:020000040800F2
:10000000A005002045010008C9100008891000085B
:10001000C51000082F0C0008772100080000000020
:1000200000000000000000000000000001150008B2
:100030006D0D0008000000005111000815160008A1
:100040005F0100085F0100085F0100085F01000810
:100050005F0100085F0100085F0100085F01000800
:100060005F0100085F0100085F0100085F010008F0
:100070005F0100085F0100085F0100085F010008E0
:100080005F0100085F0100085F0100085F010008D0
:100090005F0100085F0100085F010008710D0008A2
:1000A0005F0100085F0100085F0100085F010008B0
:1000B000211A0008591A0008211B00085F010008D6
:1000C0005F0100085F0100085F0100085F01000890
:1000D0005F010008E11E00085F0100085F010008E1
:1000E0005F0100085F0100085F0100085F01000870
:1000F0005F0100085F0100085F0100085F01000860
:100100005F0100085F010008591B00085F0100083B
:100110005F0100085F0100085F0100085F0100083F
:100120005F0100085F0100085F0100085F0100082F
:10013000DFF80CD000F008FD00480047F92A00085D
:10014000A00500200648804706480047FEE7FEE776
:10015000FEE7FEE7FEE7FEE7FEE7FEE7FEE7FEE777
:100160001916000831010008D2B201E000F8012B95
:10017000491EFBD270470022F6E710B513460A4627
:1001800004461946FFF7F0FF204610BD10B50022C7
:1001900000E0521C835C8C5CA34201D1002BF8D19F
:1001A000D8B2E1B2401A10BD70B50F4D00B9286841
:1001B000002412E00A4602E09E4203D0521C13784B
:1001C000002BF9D1DAB2224305D02BB124B10021A2
:1001D00000F8011B04E00446401C0678002EE9D11B
:1001E0002860204670BD00004800002070B506461B
:1001F00001F0D4FF046805460A220021304600F0D1
:100200006DFB2C6070BDF0B480EA0102D40F420097
:10021000B2EB410F02D20246084611464A0042D0D4
:10022000C30DDDB2C1F3C752AD1A202D35DAC1F3CB
:10023000160141F4000204B15242C5F1200602FA4F
:1002400006F12A411044B3EBD05F23D0C4B1012D95
:10025000A0EBC35009DCF0BC4FF0004202EAC352ED
:10026000DBB200F5000000F07ABB400000F18070C6
:1002700000EBC350A0F1807040EAD170490009E062
:10028000490841EAC071A0EBC35000F500004008E6
:1002900000EBC350F0BC00F059BB6142012202EBFD
:1002A0004101001BF6E7F0BC704781F00041AAE76E
:1002B00080F00040A7E780EA010210B502F0004399
:1002C000400022D04A001FD0010E01EB1261C0F3A2
:1002D0005600C2F3560240F4000042F40002A0FBB4
:1002E000022000047F39140400D0401C50EA124060
:1002F00001D44000491EC2B20C0604EBD010401CD1
:100300004008802A02D003E0002010BD20F0010048
:10031000002900DA0020184310BD30B480EA010241
:1003200002F0004530F0004221F0004013D090B1BF
:10033000C30DD40DC2F31601C0F31600E41A41F444
:10034000000140F400027D34914201D3641C00E0BE
:100350004900002C02DA30BC002070474FF4000046
:100360000023914201D3891A034340084FEA410117
:10037000F7D151B1914202D14FF0004105E002D2D4
:100380004FF0010101E06FF0010103EBC45028447C
:1003900030BC00F0DBBA2DE9FE4F804681EA030055
:1003A000C00F0C46009021F0004123F00045B8EB4F
:1003B0000200A94105D24046214690461C460B4604
:1003C000024623F00040104347D0270DC7F30A0030
:1003D000C3F30A510290401A019040286BDAC3F32C
:1003E000130040F4801B0098924620B10023D2EB0A
:1003F000030A63EB0B0B01985946C0F140025046CB
:1004000000F03BFA06460D4650465946019A00F068
:1004100053FA10EB08006141002487EA115284EA84
:10042000E7731A4340D0009A62B3019A012A4FEA57
:10043000075215DC001B61EB02014FF0004202EA9B
:100440000752CDE90042001C41F5801132462B468F
:1004500000F0C2FA03B0BDE8F08F40462146F9E74C
:10046000001B61EB0201001C41F5801300185B4189
:100470002018A2F5001747EB030140EAD570B61922
:100480006D4111E06D084FEA360645EAC0754FEA46
:100490000752001B61EB0201001C41F58011490865
:1004A0004FEA30000019514132462B4603B0BDE8F7
:1004B000F04F00F082BA0098012240000023D0EBF8
:1004C000020263EBE073009821464FEAE074B8EB58
:1004D000000061EB0401E9E783F000435BE781F092
:1004E000004158E72DE9FE4F81EA030404F000447F
:1004F00021F0004100944FF0000B23F0004350EA3C
:1005000001045ED052EA03045BD0C3F30A54C1F382
:100510000A552C44A4F2F3340194A0FB0254C1F315
:10052000130141F48011C3F3130343F4801301FB5F
:10053000024400FB034E840A970A44EA815447EAC6
:100540008357A4FB076802958D0A05FB07854FEAD0
:10055000932C04FB0C542705029D4FEA065847EAEA
:100560001637B5EB08056EEB070C870E920E47EABF
:10057000811742EA8312A7FB0201B6EB0B0164EB81
:1005800000042B0D43EA0C335E1844EB1C50DA4692
:100590005146E7FB0201C5F313044FEA0B3343EA6C
:1005A00014534FEA0432019C43EA0603A4F10C04FD
:1005B0000294009CCDE900B400F00EFA03B0BDE84F
:1005C000F08F00200146F9E72DE9F04D81EA0304A0
:1005D00004F0004B21F0004514464FF0000A23F0D0
:1005E000004150EA050220D054EA01021DD0C5F3B3
:1005F0000A570246C5F31303C1F31300C1F30A56A9
:1006000040F4801543F48013A7EB0608101BD64670
:1006100008F2FD3873EB050002D308F1010801E090
:1006200092185B41B8F1000F03DA00200146BDE8E3
:10063000F08D00204FF48011064684460EE0171B13
:1006400073EB050705D3121B63EB050306434CEA66
:10065000010C49084FEA300092185B4150EA01074B
:10066000EDD152EA030012D082EA040083EA0501C8
:10067000084305D0101BAB4106D20122002306E03F
:1006800000224FF0004302E06FF0010253101AEB1A
:1006900006004CEB085110EB0A0041EB0B01BDE8E2
:1006A000F04D00F08AB9C10F80EAE0700844CA0733
:1006B0009623002100F053B996230022114600F042
:1006C0004EB90EB5C10F80EAE0700844CA07002198
:1006D00040F233438DE80E000A460B4600F07CF9E9
:1006E00003B000BD20F00040C10DC0F3160040F47F
:1006F00000007F2901DA00207047962903DCC1F150
:100700009601C840704796398840704770B5C1F36C
:100710000A5201F000450024C1F3130140F2FF33F7
:1007200041F480119A4201DA002070BD40F2334357
:100730009A42A2F2334203DC524200F0ADF800E0EC
:1007400090402C43F1D0404270BD00F0004230F0A8
:1007500000400AD0C10D01F56071C0F3160042EAF5
:100760000151C208400711437047002001467047FD
:1007700030B5041E71F1000404DB4FF00044404228
:1007800064EB0101141E73F1000405DB1C464FF0FD
:100790000043524263EB0403994208BF904230BDCC
:1007A00001F0004330B421F0004150EA010206D0CC
:1007B0000A0DA2F56072C1F31301002A02DC30BCFD
:1007C00000207047440F44EAC104C100E01830BC67
:1007D00000EBC25000F0BAB8002801DBC0F10040C5
:1007E000002901DBC1F100418142704730B50B4661
:1007F000014600202022012409E021FA02F59D4251
:1008000005D303FA02F5491B04FA02F52844151E24
:10081000A2F10102F1DC30BD2DE9F05F05460020B8
:1008200092469B4688460646814640241BE0284661
:1008300041464746224600F02FF853465A46C01A12
:10084000914110D311461846224600F016F82D1A91
:1008500067EB01084F4622460120002100F00DF809
:1008600017EB00094E41201EA4F10104DFDC4846CD
:1008700031462A464346BDE8F09F202A04DB203A51
:1008800000FA02F1002070479140C2F1200320FAE3
:1008900003F3194390407047202A04DB203A21FAE1
:1008A00002F00021704721FA02F3D040C2F1200289
:1008B0009140084319467047202A06DBCB17203A9F
:1008C00041FA02F043EAE07306E041FA02F3D04055
:1008D000C2F1200291400843194670472DE9F047C4
:1008E00091460F4680460446002614F8015B2DB160
:1008F00000F03CF90068405DC007F6D12B2D02D016
:100900002D2D18D0641E4A463946204600F032F993
:1009100027B13968A14201D1C7F8008071054FF0B5
:1009200002040BD54042002803DD01F037FC0460CF
:10093000A007BDE8F08746F48066E4E70028F8DA0F
:1009400001F02CFC04606FF00040F2E70029A8BF22
:100950007047401C490008BF20F00100704710B4E8
:10096000B0FA80FC00FA0CF050EA010404BF10BC9D
:10097000704749B1CCF1200421FA04F411FA0CF1CA
:1009800018BF012121430843A3EB0C01CB1D4FEA03
:1009900000614FEA102042BF002010BC704700EBFE
:1009A000C35010440029A4BF10BC7047401C49002C
:1009B00008BF20F0010010BC704710B5141E73F181
:1009C000000408DA401C41F1000192185B411A430F
:1009D00001D120F0010010BD2DE9F04D92469B465B
:1009E00011B1B1FA81F202E0B0FA80F22032904601
:1009F000FFF743FF04460F4640EA0A0041EA0B01B5
:100A000053465A46084313D0114653EA010019D001
:100A1000C8F140025046FFF73FFF05460E465046DC
:100A200059464246FFF729FF084305D0012004E05C
:100A300020463946BDE8F08D0020054346EAE076C1
:100A40002C4337430A986305E40AA0EB0800002210
:100A5000FD0A44EA47540A3002D500200146E9E77E
:100A6000010510196941DDE9084500196941BDE832
:100A7000F04DA2E72DE9F04D00231A461B1A8A41DA
:100A800003DB00200146BDE8F08DC1F30A52C1F33B
:100A9000130141F480154FF0000BD10702D100186B
:100AA0006D41521E0027044640F2FF11384601EB0B
:100AB000620A3E468046024600204FF48011FFF74E
:100AC000EBFEC2197141BB1846EB0100B4EB030CFD
:100AD00075EB000C04D3E41A65EB000517460E46CF
:100AE000241908F101006D4180463428E3DDF9192D
:100AF00046EB0600091BA84103D24FF0FF32134614
:100B000001E0002213461BEB070046EB0A51BDE84B
:100B1000F04DFFF752BFC1F30A52C1F3130140F287
:100B2000FF3341F480119A4202DA002001467047F7
:100B300040F233439A42A2F2334202DC5242FFF7C0
:100B4000ABBEFFF79ABE0000064C074D06E0E0681A
:100B500040F0010394E8070098471034AC42F6D304
:100B6000FFF7EAFA84360008A43600080048704708
:100B7000803600082DE9F05F824600780027154690
:100B80008B460AF10104B946302801D09DB113E02B
:100B900014F8010B0127782803D0582801D045B15B
:100BA0000AE00DB1102D07D10027102514F8010B14
:100BB00002E0082500E00A250026B0460EE005FB0D
:100BC000080005FB06F1012701EB10461FFA80F82B
:100BD000B6F5803F00D3B94614F8010B294600F062
:100BE00018F80028EBDABBF1000F05D00FB1641E36
:100BF00000E05446CBF80040B9F1000F06D001F0F8
:100C0000CDFA02210160C81EBDE8F09F48EA064007
:100C1000FAE73A2800D2303820F02002412A01D3E6
:100C2000A2F13700884201D34FF0FF30704700BF78
:100C3000FEE7000039B1084A1268012383401A43D5
:100C4000054B1A6006E0044A1268012383409A4368
:100C5000014B1A60704700000074004030B500225C
:100C600000230A4C226840F6FE748440A243D1E976
:100C700000452C438D682C43CD6844EA050303FAF4
:100C800000F42243014C226030BD0000007400409B
:100C900008B500220092054A009200F10802009B6C
:100CA0001A440092009A116008BD000000740040D0
:100CB00000B585B00121042000F05CFA012148074D
:100CC00000F048FA1020ADF8100000208DF8130055
:100CD00003208DF8120004A90D4800F03DF9102101
:100CE0000B4800F0CFF90020009001900290022004
:100CF000039069460020FFF7B1FF01210020FFF7B4
:100D000099FF00210846FFF7C3FF05B000BD0000B2
:100D1000000801402DE9F04704462046FFF7CCFCCF
:100D2000814610494846FFF7F8FA81464FF08B415B
:100D30004846FFF7C0FA8246FFF707FD07464FF027
:100D40006632094BFFF740FC0546FFF729FD814657
:100D50004846FFF7C7FC85B229460020FFF798FFF9
:100D6000BDE8F08700007A4466660A4070470000DC
:100D700010B5402000F072F8D0B101200D49C1F843
:100D8000800002F0D5FB0B4890F87800012809D1CB
:100D900009A001F0F3F94FF0FF3006494867002041
:100DA000086002E009A001F0E9F9402000F01AF81B
:100DB00010BD000050000020416C72656164792014
:100DC0006174205A45524F0D0A000000616C726533
:100DD00061647920636C6F736520262066750D0A47
:100DE0000000000001490860704700001404014041
:100DF0001FB50121082000F0BDF94020ADF80C001E
:100E000004208DF80F0003A9134800F0A5F8012174
:100E1000084600F0AFF90621012000F07DF84020DF
:100E2000019000208DF8080008208DF809000120AD
:100E30008DF80A0001A800F025F817208DF80000B1
:100E400000208DF801008DF8020001208DF80300CC
:100E5000684600F03BF91FBD000C01400146002030
:100E60000022074B1B6803EA0102054B14331B6881
:100E70000B4013B10AB1012000E0002070470000D0
:100E800000040140002123498279002A3AD00A4611
:100E9000126803689A430B461A600A1D12680368B9
:100EA0009A430B1D1A60027911440A6803681A43B9
:100EB0000A60184A0832126803689A43154B0833CF
:100EC0001A601A1D126803689A43124B0C331A6099
:100ED0004279102A0ED11A1F126803681A430D4B6B
:100EE00008331A601A1D126803681A43094B0C3341
:100EF0001A600DE00749427911440A6803681A43F1
:100F00000A6005E0027911440A6803689A430A609E
:100F1000704700000004014030B500228B071C0F11
:100F20000F2303FA04F20B4B8C1053F82430934335
:100F3000084C8D1044F8253023468C1053F824308B
:100F40008C07240F00FA04F42343024C8D1044F85C
:100F5000253030BD080001402DE9F0410246002552
:100F60000026002000230024002791F803C00CF085
:100F70000F0591F803C00CF0100CBCF1000F03D06A
:100F800091F802C04CEA050591F800C0BCF1000FD1
:100F900031D0146800202BE04FF0010C0CFA00F364
:100FA000B1F800C00CEA03069E4220D183004FF046
:100FB0000F0C0CFA03F7BC4305FA03FC4CEA0404DB
:100FC00091F803C0BCF1280F06D14FF0010C0CFAC8
:100FD00000FCC2F814C00AE091F803C0BCF1480F4D
:100FE00005D14FF0010C0CFA00FCC2F810C0401CF7
:100FF0000828D1D31460B1F800C0BCF1FF0F34DD74
:10100000546800202EE000F1080C4FF0010808FAA7
:101010000CF3B1F800C00CEA03069E4221D1830014
:101020004FF00F0C0CFA03F7BC4305FA03FC4CEA33
:10103000040491F803C0BCF1280F05D100F1080C9D
:1010400008FA0CF8C2F8148091F803C0BCF1480FFC
:1010500007D100F1080C4FF0010808FA0CF8C2F8AB
:101060001080401C0828CED35460BDE8F0810246B1
:10107000002093680B400BB1012000E00020704776
:10108000416170470161704700BFFEE708B501216B
:10109000082000F06FF84FF48050ADF800001020E9
:1010A0008DF8030003208DF8020069460448FFF71D
:1010B00053FF4FF480510248FFF7E4FF08BD0000E2
:1010C000000C014000BFFEE77047000070B5002132
:1010D00000230F22C47804B3154C246804F4E064A0
:1010E000C4F5E064210AC1F10403CA40447804FA5B
:1010F00003F184781440214309010E4C0678A15570
:10110000047804F01F050124AC4005786D11AD0092
:1011100005F1E025C5F8004109E0047804F01F0559
:101120000124AC40044D0678761145F8264070BD88
:101130000CED00E000E400E080E100E00249014342
:10114000024A1160704700000000FA050CED00E053
:101150007047000029B1064AD2690243044BDA61A4
:1011600004E0034AD2698243014BDA617047000010
:101170000010024029B1064A92690243044B9A6169
:1011800004E0034A92698243014B9A617047000070
:101190000010024030B500210022002400232D4D14
:1011A0006D6805F00C0121B1042905D0082923D16F
:1011B00005E0294D056022E0274D05601FE0254D23
:1011C0006D6805F47012234D6D6805F480340225B6
:1011D00005EB92421CB9214D554305600BE01D4DB6
:1011E0006D6805F400351DB11C4D5543056002E0E6
:1011F000194D5543056002E0174D056000BF00BF63
:10120000144D6D6805F0F0010909154D6B5C05681A
:10121000DD4045600F4D6D6805F4E061090A104D31
:101220006B5C4568DD4085600A4D6D6805F4605172
:10123000C90A0B4D6B5C4568DD40C560054D6D68A6
:1012400005F44041890B074D6B5CC568B5FBF3F5B0
:10125000056130BD0010024000127A0000093D0017
:10126000340000204400002010B54FF4805106489F
:10127000FFF708FF01200549086148600020C860A9
:1012800001200349086010BD000801405000002003
:101290000400002010B54FF400610448FFF7F2FE8F
:1012A0004FF47A70FFF736FD10BD000000080140D2
:1012B00010B54FF480510648FFF7E2FE01200549C2
:1012C000086100204860C86001200349086010BD23
:1012D00000080140500000200000002008B5012156
:1012E0001C20FFF747FF41F61010ADF8000010205A
:1012F0008DF8030003208DF8020069460F48FFF7C0
:101300002BFE4FF46040ADF8000010208DF8030074
:1013100003208DF8020069460948FFF71DFE0120F1
:10132000ADF8000010208DF8030003208DF80200B6
:1013300069460448FFF710FE08BD000000080140A0
:10134000000C01400010014010B500200749086161
:101350004FF400610648FFF793FE06A000F00EFF71
:1013600000214FF40060FFF705FF10BD5000002082
:1013700000080140414C52454441595F4F46464C9C
:10138000494E450D0A00000010B50121C802FFF7C3
:10139000F1FE10BD10B50446102C58D008DC012C0D
:1013A0000DD0022C1ED0042C2ED0082C72D13DE082
:1013B000202C5ED0402C6FD0802CF7D17DE0002215
:1013C0004FF40051484802F07DF800224FF480416C
:1013D000454802F077F800224FF40041424802F0FD
:1013E00071F87FE0012251033F4802F06BF80022C0
:1013F0004FF480413C4802F065F800224FF4004170
:10140000394802F05FF86DE000224FF40051364891
:1014100002F058F801229103334802F053F80022F9
:101420004FF40041304802F04DF85BE001225103D7
:101430002D4802F047F8012291032B4802F042F8B0
:1014400000224FF40041284802F03CF84AE0002214
:101450004FF40051244802F035F800224FF4804147
:10146000214802F02FF80122D1031F4802F02AF888
:1014700038E0012251031C4802F024F801229103B4
:10148000194802F01FF800224FF40041164802F0FC
:1014900019F827E021E0FFE700224FF4005112483D
:1014A00002F010F8012291030F4802F00BF801221C
:1014B000D1030D4802F006F814E0012251030A4856
:1014C00002F000F801229103074801F0FBFF01221E
:1014D000D103054801F0F6FF04E0214603A000F027
:1014E0004DFE00BF00BF10BD000C01404572726F81
:1014F000722076616C75653A2025640D0A00000043
:10150000704710B500F002F810BD00000CB50020C7
:10151000019000903348006840F480303149086001
:1015200000BF3048006800F4003000900198401C73
:101530000190009818B90198B0F5A06FF1D1294831
:10154000006800F4003010B10120009001E000209C
:1015500000900098012843D12348006840F0100013
:10156000214908600846006820F00300086008462A
:10157000006840F0020008601A4840681949486055
:101580000846406848600846406840F4806048600B
:101590000846406820F47C1048600846406840F4E3
:1015A000E81048600846006840F08070086000BF9E
:1015B0000C48006800F000700028F9D00948406825
:1015C00020F00300074948600846406840F00200E8
:1015D000486000BF0348406800F00C000828F9D1BB
:1015E0000CBD00000010024000200240042808D179
:1015F0004FF0E021096941F004014FF0E022116150
:1016000007E04FF0E021096921F004014FF0E022EA
:10161000116170477047000010B51348006840F032
:1016200001001149086008464068104908400E4909
:101630004860084600680E4908400B4908600846A3
:10164000006820F4802008600846406820F4FE000E
:1016500048604FF41F008860FFF753FF4FF00060B1
:101660000449086010BD0000001002400000FFF8AF
:10167000FFFFF6FE08ED00E0F0B50C46154600222F
:101680000021068C4FF6FE773E400684028B018CCB
:101690004FF60C7632407E1C06EA03162E43324388
:1016A000104EB0420ED0104EB0420BD0B0F1804F71
:1016B00008D00E4EB04205D00D4EB04202D00D4EB5
:1016C000B04206D14FF6FD76314044F00106314379
:1016D00005E04FF6F576314044F0010631430283D0
:1016E0000184F0BD002C01400034014000040040A2
:1016F00000080040000C0040F0B50C4615460022E2
:1017000000210026078C4FF6EF7C07EA0C070784C0
:10171000028B018C4FF6FF7707EA041640F6FF476D
:101720003A404FF6FF7707EA03373A434FF6FF7721
:1017300007EA05273A43114FB8420ED0104FB8427E
:101740000BD0B0F1804F08D00E4FB84205D00E4FED
:10175000B84202D00D4FB84206D14FF6DF7739407C
:1017600046F01007394305E04FF65F77394044F003
:101770001007394302830184F0BD0000002C0140B2
:10178000003401400004004000080040000C00400C
:10179000F0B50C461546002200210026078C4FF6B6
:1017A000FF6C07EA0C070784828B018C4FF6FF77EA
:1017B00007EA04264FF60C773A404FF6FF7707EA20
:1017C00003172F433A43114FB8420ED0104FB8427F
:1017D0000BD0B0F1804F08D00E4FB84205D00E4F5D
:1017E000B84202D00D4FB84206D14FF6FF573940EC
:1017F00046F48077394305E04FF2FF57394044F40F
:101800008077394382830184F0BD0000002C0140C1
:10181000003401400004004000080040000C00407B
:10182000F0B50C461546002200210026078C4EF626
:10183000FF7C07EA0C070784828B018C4FF6FF7749
:1018400007EA043640F6FF473A404FF6FF7707EACB
:1018500005273A434FF6FF7707EA03373A43114F1C
:10186000B8420ED0104FB8420BD0B0F1804F08D024
:101870000E4FB84205D00E4FB84202D00D4FB842BD
:1018800006D14DF6FF77394046F48057394305E0DD
:1018900047F6FF57394044F4805739438283018427
:1018A000F0BD0000002C0140003401400004004065
:1018B00000080040000C004000B589B00121C802BA
:1018C000FFF758FC01210420FFF754FC18208DF885
:1018D00023004FF48070ADF8200003208DF8220023
:1018E00008A92448FFF738FB234800F012FA00202B
:1018F000ADF81A00ADF8160040F2E730ADF8180068
:101900004720ADF8140000208DF81C0005A91A48E6
:1019100000F094FA01A800F04FFA7020ADF804002E
:101920000020ADF80C000120ADF8060042F2107066
:10193000ADF80A0001A9104800F0F2F901210E48A3
:1019400000F068F901210C4800F046F920210A480E
:1019500000F03CFA0121084800F04AF90122114642
:10196000054800F0CDF90121034800F047F909B01E
:1019700000BD000000080140002C014000B589B006
:1019800001210846FFF7E6FB0120ADF820004820C2
:101990008DF8230003208DF8220008A91F48FFF7C7
:1019A000DBFA4FF6FF70ADF818004720ADF81400D1
:1019B0000020ADF81A00ADF8160005A94FF08040E0
:1019C00000F03CFA0020ADF80800ADF80A00012054
:1019D000ADF80C000020ADF80E00ADF8100002A923
:1019E0004FF0804000F036F91C208DF804000020F4
:1019F0008DF805008DF8060001208DF8070001A87C
:101A0000FFF764FB01220221480700F079F9012168
:101A1000880700F0F3F809B000BD0000000801409D
:101A200010B50221480700F004F940B101F080FD33
:101A300003A000F0A3FB0221480700F0DCF810BD72
:101A4000616C726561647920636C6F736520262018
:101A50007A68656E670D0A0010B50221044800F02F
:101A6000E8F818B10221024800F0C5F810BD0000E6
:101A70000004004030B589B004460D460121022023
:101A8000FFF768FB4720ADF814000020ADF8160002
:101A90004FF6FF70ADF818000020ADF81A0005A948
:101AA0001D4800F0CBF90020ADF804000A20ADF885
:101AB00006000120ADF808000020ADF80A00ADF8DE
:101AC0000C0001A9144800F0C5F84020ADF8200032
:101AD00028208DF8230003208DF8220008A90F4844
:101AE000FFF73AFA1D208DF8100000208DF8110044
:101AF00003208DF8120001208DF8130004A8FFF7D1
:101B0000E5FA0121044800F079F801220221024897
:101B100000F0F6F809B030BD0004004000080140B4
:101B200010B50221054800F084F830B104A000F09F
:101B300025FB0221014800F05EF810BD00080040BE
:101B4000616C726561647920636C6F736520262017
:101B500066750D0A0000000010B50121064800F06E
:101B600068F838B100F0AEFF01F06AFA01210248CE
:101B700000F041F810BD0000000C00407FB50546A4
:101B80000C4601210820FFF7E5FAADF80850ADF842
:101B900004400020ADF80A00ADF8060001A90D4888
:101BA00000F04CF9012211460A4800F0A9F8322051
:101BB0008DF8000000208DF8010001208DF8020052
:101BC0008DF803006846FFF781FA0121014800F013
:101BD00015F87FBD000C004021B1028842F0800260
:101BE000028004E002884FF67F731A40028070473B
:101BF000CA4302827047CA430282704721B10288F9
:101C000042F00102028004E002884FF6FE731A409F
:101C10000280704731B1B0F8442042F40042A0F88D
:101C2000442005E0B0F84420C2F30E02A0F844209E
:101C3000704730B50246002000230024158A05EACB
:101C40000103958905EA010413B10CB1012000E0FC
:101C5000002030BD70B505460C46244885420ED0A4
:101C6000234885420BD0B5F1804F08D021488542EA
:101C700005D02148854202D02048854200D100E0AD
:101C800000BF208850B92389A28861882846FFF7C1
:101C9000F3FCE188284600F0A4F825E02088042819
:101CA0000AD12389A28861882846FFF725FDE188AB
:101CB000284600F09FF817E0208808280AD12389D9
:101CC000A28861882846FFF763FDE188284600F076
:101CD0009EF809E02389A28861882846FFF7A0FDC5
:101CE000E188284600F09CF870BD0000002C0140FF
:101CF000003401400004004000080040000C004097
:101D00001AB183890B43838102E083898B438381EA
:101D1000704701894FF6F872114001817047000049
:101D200070B5002400220023058C4FF6FE76354066
:101D30000584028C8388048B4FF68F752C40B51E6A
:101D40002C400D882C43751E2A400D892A434D884E
:101D50002A43144DA8420BD0134DA84208D0134D6E
:101D6000A84205D0124DA84202D0124DA84213D16C
:101D70004FF6F7752A404D892A434FF6FB752A40E6
:101D80008D882A434FF6FF652B404FF6FF552B40B9
:101D90008D892B43CD892B4383800483CD88858611
:101DA000028470BD002C014000340140004001401D
:101DB00000440140004801400021018041808180B1
:101DC000C180018141818181C181704782884FF644
:101DD0008F731A40828082880A438280704781868E
:101DE0007047028B4FF6F3731A400283028B0A434B
:101DF00002837047028B4FF2FF331A400283028B3B
:101E00004FF6FF7303EA01231A4302837047828B64
:101E10004FF6F3731A408283828B0A4382837047A2
:101E2000828B4FF2FF331A408283828B4FF6FF730F
:101E300003EA01231A4382837047000000220288CC
:101E40001D4B98420ED01D4B98420BD0B0F1804FE5
:101E500008D01B4B984205D01A4B984202D01A4B1F
:101E6000984204D14FF68F731A404B881A43174B90
:101E7000984207D0164B984204D04FF6FF431A40C1
:101E8000CB881A4302808B8883850B8803850A4B95
:101E900098420BD0094B984208D00E4B984205D07F
:101EA0000D4B984202D00D4B984201D10B7A03861C
:101EB0000123838270470000002C01400034014060
:101EC0000004004000080040000C004000100040EA
:101ED000001400400040014000440140004801401F
:101EE00010B540F22551264800F081F838B340F291
:101EF0002551234800F053F8214800F033F9C4B2CB
:101F00002048008800F40040C8B91E48008800F44A
:101F1000804060B10A2C03D000201A49088020E0DC
:101F20001848008840F400401649088019E00D2C3C
:101F300006D11448008840F480401249088010E01F
:101F400010480088C0F30D000F490C540D4800885C
:101F5000401C0C49088008460088C72801DD002085
:101F600008800821064800F035F8012806D108212C
:101F7000034800F00BF8024800F0F4F810BD000030
:101F8000003801402C000020D800002001F400722D
:101F9000B2F5007F00D100BFCA430280704710B580
:101FA0000022002340F66A14A14200D100BF0A12A9
:101FB00001249440A3B2DC43048010BD21B1828986
:101FC00042F40052828104E082894DF6FF731A4088
:101FD0008281704702460020B1F5007F00D100BF2A
:101FE00013880B400BB1012000E00020704770B552
:101FF0000246002400230025002040F66A16B14264
:1020000000D100BFC1F3421501F01F03012606FAFB
:1020100003F3012D02D19689334006E0022D02D14F
:10202000168A334001E0968A33400C12012606FAE4
:1020300004F41688344013B10CB1012000E00020F4
:1020400070BDF0B50346002400260025002040F6B0
:102050006A17B94200D100BF1846C1F3421401F01B
:102060001F06012707FA06F5012C01D10C3004E008
:10207000022C01D1103000E014301AB107682F4350
:10208000076002E00768AF430760F0BD2DE9F04745
:1020900086B005460E460024A24600BFA146002792
:1020A000B08900B100BF2F462C8A4CF6FF70044067
:1020B000F08804432C82AC894EF6F3100440B088BB
:1020C00031890843718908430443AC81AC8A4FF6D7
:1020D000FF400440B0890443AC8201A8FFF75AF8DE
:1020E0001F48874202D1DDF810A001E0DDF80CA006
:1020F000A88900F4004040B10AEBCA0000EB0A10C6
:1021000031684900B0FBF1F807E00AEBCA0000EBC8
:102110000A1031688900B0FBF1F86420B8FBF0F0D8
:1021200004012009642101FB1089A88900F4004002
:1021300040B1322000EBC900B0FBF1F000F0070025
:10214000044308E0322000EB09106421B0FBF1F0F9
:1021500000F00F0004432C8106B0BDE8F0870000BA
:102160000038014001468888C0F308007047C1F379
:1021700008028280704700BFFEE700000FB4054BE5
:1021800010B503A9044A029800F0D4F810BC5DF819
:1021900014FB0000A92A000828000020004870470E
:1021A0004C00002002E008C8121F08C1002AFAD122
:1021B00070477047002001E001C1121F002AFBD1C7
:1021C0007047000001490860704700004C00002083
:1021D0002DE9FF5FDDE90220010DDDF838B0024393
:1021E00018D044F61050A1F2FF3141430D140F985E
:1021F000012820D0A5EB0B00401C5FEA000A4FF03D
:102200000004474EDFF81C91A046504616D5CAF18F
:10221000000728E00F98012443A2012808D00021DC
:1022200000980F9BC0E90021C0E90243BDE8FF9F71
:102230006FEA0B01F4E7CBF10000DEE7074612E09E
:10224000F80707D02246334640464946FEF74AF98A
:10225000804689462246334610461946FEF742F923
:1022600004460E467F10002FEAD1DDE90201BAF1E3
:10227000000F42464B4602DAFEF734F901E0FEF762
:10228000A3F904460E460022284BFEF771FA03D844
:102290004FF0FF30014607E00022254B2046314633
:1022A000FEF779F8FEF737FC102409E0002C0ADB72
:1022B0000A220023FEF7B0FA019B30321A55641E41
:1022C00050EA0102F2D1641C019AC4F111031444D2
:1022D0000F9A012A03D0012208430DD10AE00843D6
:1022E00004D000204FF0110B0F9080E7A3EB0B05FB
:1022F0006D1E0DE05B4504DD4FF0000205F10105A8
:1023000004E003DA4FF00002A5F10105002AECD049
:1023100000980F99C0E90231C0E9004586E7000046
:10232000000024400000F03F300000000000F043B7
:102330000000E03F2DE9FF4F95B09B4689460646D9
:1023400000250FE2252877D100242746F84A0121ED
:10235000059400E0044316F8013F203B01FA03F026
:102360001042F7D130782A2811D06FF02F0330783F
:10237000A0F13002092A16D8059A44F0020402EBB3
:10238000820203EB42021044761C0590EFE759F8F5
:10239000042B0592002A03DA504244F400540590BD
:1023A00044F00204761C30782E2816D116F8010F5E
:1023B00044F004042A280DD06FF02F023078A0F1E9
:1023C0003003092B09D807EB870302EB4303C71837
:1023D000761CF3E759F8047B761C30786C280FD014
:1023E00006DC4C2817D068280DD06A2814D104E0E8
:1023F000742810D07A280FD10DE044F400140AE0BC
:1024000044F4801401E044F440147278824202D112
:1024100004F58014761C761C307866280BD013DC0B
:10242000582877D009DC002875D04528F6D04628F2
:10243000F4D047281AD19DE118E0632835D06428EC
:1024400079D0652812D195E1702873D008DC67280F
:10245000F1D069286FD06E280DD06F2806D1B5E075
:1024600073282CD0752875D0782874D05A461799BF
:1024700090476D1C75E1C4F30250022809D003286F
:102480000DD0D9F8001004280DD00D6009F1040911
:1024900067E1D9F80010EA17C1E90052F6E7D9F868
:1024A00000100D80F2E70D70F0E719F8041B8DF8AD
:1024B000001000208DF80100EA46012003E059F8E1
:1024C00004AB4FF0FF3061074FF0000102D40DE084
:1024D00008F101018846B9420FDA8045F8DB1AF8A5
:1024E00008100029F4D108E008F101018846814272
:1024F000FADB1AF808100029F6D105985B46A0EB24
:10250000080721463846179A00F094FA284400EB51
:10251000080507E04DE029E10DE01AF8010B5A46E5
:1025200017999047B8F10108F7D25B462146384623
:10253000179A13E142E00A220092C4F302524FF0CC
:10254000000A022A08D059F804CB032A4FEAEC719A
:102550000AD00DE029E02AE009F1070121F0070285
:10256000F2E802C1914609E00FFA8CFC4FEAEC71E7
:10257000042A03D14FFA8CFC4FEAEC71002907DAE8
:102580000A460021DCF1000C61EB02012D2202E081
:10259000220504D52B228DF80420012203E0E20756
:1025A00001D02022F7E7904659E00A2102E01022EC
:1025B0000DE010214FF0000A00910BE010224FF0C7
:1025C000000A44F004040827009203E008224FF0B8
:1025D000000A0092C4F30252022A05D059F804CB33
:1025E0000021032A08D009E009F1070121F00702C0
:1025F000F2E802C1914605E01FFA8CFC042A01D1E1
:102600000CF0FF0C4FF00008220728D5702806D0E8
:10261000009B83F0100353EA0A0305D00EE040222A
:102620008DF80420012208E05CEA010206D0302285
:102630008DF804208DF8050002229046009B83F05F
:10264000080353EA0A030AD15CEA010201D16207D6
:1026500005D530228DF804204FF001087F1E582840
:1026600004D034A003900EA802900DE036A0F9E744
:1026700053466046009AFEF7CFF884460398825C82
:102680000298401E029002705CEA0100F0D10298AC
:1026900006A9081A00F1200A600702D524F4803444
:1026A00000E00127574502DDA7EB0A0000E000200B
:1026B00000EB0A01009005984144401A0590E003A0
:1026C00006D45B462146179A059800F0B3F90544F5
:1026D000002706E001A85A46C05D179990476D1C77
:1026E0007F1C4745F6DBE0030CD55B462146179A75
:1026F000059800F09FF9054404E030205A461799E8
:1027000090476D1C0099481E00900029F5DC08E0F8
:10271000029802995A460078491C029117999047ED
:102720006D1CBAF10001AAF1010AF1DC65E10000BB
:102730000928010030313233343536373839616297
:10274000636465660000000030313233343536375B
:1027500038394142434445460000000000F058F932
:102760000544761C307800287FF4ECAD19B028467B
:10277000BDE8F08F620700D4062709F1070222F0B6
:10278000070CFCE80223E14603F000485FEA080C6E
:1027900002D00FF2702C0DE05FEA045C02D50FF25C
:1027A000682C07E05FEAC47C02D00FF2602C01E0E5
:1027B000AFF2700C4FF0FF3823F00043CDF850C05B
:1027C00065280CD006DC452809D046281DD04728AE
:1027D0003DD13DE0662818D067287ED138E0002141
:1027E000112F01DB112000E0781CCDE9000106A9C2
:1027F0000EA8FFF7EDFCDDE90F010E9A0391002111
:10280000009207F1010A04914DE04FF0004000975B
:10281000CDE9011006A90EA8FFF7DAFCDDE90F02E9
:1028200003920E9B11990022DDF80CA000930492F4
:1028300011B9791C00EB010AB7EB0A0004D4C0F10E
:10284000FF3007F1010A0490AAEB0700019044E071
:10285000012F00DA01270021112F01DD112000E0F6
:102860003846CDE9000106A90EA8FFF7B1FCDDE965
:102870000F010E9A0391002104910092BA4621079C
:102880000CD40399514500DA8A46BAF1010F05DDEF
:10289000009AAAF10101515C302908D0B84202DA4D
:1028A00010F1040F06DA0121CDE9011015E0AAF1BB
:1028B0000101E9E7002805DC049901440491AAEB31
:1028C000000102E0411C514500DD8A460499401A8E
:1028D000401C01904FF000400290200704D4019862
:1028E000504501DBCDF8048000208DF84F000298A0
:1028F0000DF14F07B0F1004F25D02B200E9002981C
:102900004FF0020800280CDA404202902D200E9071
:1029100007E00A210298FDF769FF3031029007F8BD
:10292000011DB8F10001A8F10108F2DC02980028AD
:10293000EFD1791E0E980870307800F0200040F03A
:10294000450007F8020D12A8C01B00F107081498F3
:10295000007800B1012000EB0A01019801EBE07161
:1029600005984144401A401E0590E00306D45B469A
:102970002146179A059800F05DF8054414980078F0
:1029800018B15A46179990476D1CE00324D55B4651
:102990002146179A059800F04DF805441CE004986C
:1029A000002807DBDDE90301884203DD0098405C75
:1029B000179901E0179930205A469047049805F17D
:1029C0000105401C04900198401E019004D12E2066
:1029D0005A46179990476D1CBAF10001AAF1010AF5
:1029E000DDDC05E017F8010B5A46179990476D1C7E
:1029F000B8F10001A8F10108F4DC5B462146179A02
:102A00000598ABE62D0000002B0000002000000020
:102A10002DE9F041044600251E461746880404D4DB
:102A200005E039462020B0476D1C641EF9D52846C4
:102A3000BDE8F0812DE9F041044600251E46904690
:102A4000C80301D5302700E02027880404D505E01D
:102A500041463846B0476D1C641EF9D52846BDE88E
:102A6000F081000010B56FF00400FEF7BFFD0A48CA
:102A700000680A49B0FBF1F009490870084600787F
:102A800000EB4001C1EBC0104FF6FF7101EAC0003E
:102A90000449088010BD00000800002000127A00E0
:102AA000240000202600002000BF054A128802F002
:102AB0004002002AF9D0C2B2014B1B1D1A80704798
:102AC000003801400A480068401C0949086008466F
:102AD0000068C8280ADD0748006808B9012000E03E
:102AE0000020044908600020014908607047000088
:102AF00030000020B08121421CB50020E249C860AE
:102B000008600A469062D0624860886048618861C7
:102B100008610863C8614863DC480864DC484864AD
:102B200000208865401E48670020C867C1F8800003
:102B3000C86481F878004FF4FA608865FFF792FF67
:102B40004FF4A060FEF7FAFA4FF4E13000F006FD12
:102B5000FEF7C4FBFEF79AFAFEF7AEFE472140F2FD
:102B6000E730FEF787FFFEF709FFFEF741F94FF464
:102B7000FA71C848FFF733F9FEF79AF80121C64801
:102B8000FEF780FA4FF40061C448FEF779FA04209A
:102B9000FEF700FC40F2DC50FEF7BCF8C0A0FFF7E7
:102BA000EDFA70E1C448008800F400400028F8D035
:102BB000C1480088C0F30D0600250DE0BF48415D07
:102BC000BF48FFF7D4FA00BF4021BD48FFF702FA23
:102BD0000128F9D1681C85B2B542EFDB0020B64967
:102BE0000880B8A1B548FDF7DFFA8146B6A148468E
:102BF000FDF7CCFA00287DD1B2A1FDF7D5FA8146C8
:102C0000B2A14846FDF7C2FA20B9FEF7BDFBB1A05C
:102C1000FFF7B4FAB1A14846FDF7B8FA20B9FEF7BC
:102C200093FBAFA0FFF7AAFAAFA14846FDF7AEFAB3
:102C300020B9FEF72FFBADA0FFF7A0FAADA14846E3
:102C4000FDF7A4FA38B900208F49086000F070FC45
:102C5000AAA0FFF793FAABA14846FDF797FAC0B9CF
:102C600098A10020FDF7A0FA8146A9A14846FDF7EA
:102C70008DFA20B9FEF71CFBA6A0FFF77FFAAAA1E8
:102C80004846FDF783FA20B9FEF7EEFAA7A0FFF752
:102C900075FAABA14846FDF779FAB8B989A10020C9
:102CA000FDF782FA81464846FDF7A0FA044640F651
:102CB000B830844207DC204600F0BAFB2146A2A0CF
:102CC000FFF75CFA02E0A4A0FFF758FAA6A1484675
:102CD000FDF75CFAA8B9472140F2E730FEF74EFF56
:102CE00078A10020FDF760FA81464846FDF77EFA9C
:102CF000044600E070E06448446521469BA0FFF76D
:102D00003DFA9DA14846FDF741FA98B9472140F2A6
:102D1000E730FEF733FF6BA10020FDF745FA81464F
:102D20004846FDF763FA044657480465214693A0D8
:102D3000FFF724FA94A14846FDF728FA78B961A173
:102D40000020FDF731FA81464846FDF74FFA044668
:102D50002046FEF71FFB21468FA0FFF70FFA93A135
:102D60004846FDF713FA68B956A10020FDF71CFA92
:102D700081464846FDF73AFA0446204600F05EFBDD
:102D8000414884608BA14846FDF700FA70B94DA117
:102D90000020FDF709FA81464846FDF727FA044668
:102DA00039488465214685A0FFF7E8F986A14846A1
:102DB000FDF7ECF9002861D142A1FDF7F5F9814654
:102DC0004846FDF713FA044600213D48FFF7F6F8A0
:102DD000204600F0C3FB51E07EA14846FDF7D6F93E
:102DE00000284BD137A1FDF7DFF981467BA148468A
:102DF000FDF7CCF978B933A10020FDF7D5F981466C
:102E00004846FDF7F3F90446204600F027FA21462C
:102E100073A0FFF7B3F976A14846FDF7B7F990B96B
:102E200028A10020FDF7C0F981464846FDF7DEF9EC
:102E30000446E0171449C1E90A4000F0C1F92146EF
:102E40006CA0FFF79BF92BA14846FDF79FF920B92D
:102E500000F0CAFA6BA0FFF791F96EA14846FDF7A2
:102E600095F958B90849086FFDF76FFCCDE90001E5
:102E700005480268416F69A0FFF780F9C8210F4833
:102E8000FDF779F900BF8DE6500000203D340008C1
:102E900031350008002C01400010014000080140BD
:102EA00077656C6C636F6D20746F206D79206D6F2A
:102EB000746F720D0A2000002C000020D800002042
:102EC0000038014023000000534554004F50454E48
:102ED000000000004F50454E0D0A00004F464600CE
:102EE0004F46460D0A000000454E0000454E0D0AB3
:102EF000000000005A45524F000000005A45524F52
:102F00000D0A00004452454354494F4E0000000052
:102F1000300000004452454354494F4E20464F5222
:102F2000574152440D0A000031000000445245430D
:102F300054494F4E204241434B574152440D0A00E1
:102F400043555252454E540043555252454E54201B
:102F500025640D0A0000000043555252454E54208E
:102F60004F5645520000000044454300444543206D
:102F700025640D0A00000000414343004143432003
:102F800025640D0A000000004D4943524F5354453B
:102F90005050494E470000004D4943524F5354454D
:102FA0005050494E472025640D0A000053504545B6
:102FB00044000000544152474554000054415247D8
:102FC00045542025640D0A00424155445F52415446
:102FD000450000004D4F564500000000544F0000D2
:102FE0004D4F564520544F2025640D0A0000000027
:102FF000425900004D4F56452042592025640D0A84
:10300000000000004D4F564520544F205A45524F66
:103010000D0A0000494E464F000000002053746125
:1030200074733A2025642C20506F733A2025642C49
:103030002053706565643A20252E31660D0A000024
:103040002DE9F04756480069012811D154484068DD
:1030500028B953480068401C5149086008E05048AE
:103060004068012804D14E480068401E4C49086061
:103070004B48C06901287DD14948006908B9BDE8BD
:10308000F0874748006E401C454908660846016EB7
:1030900044A0FFF773F84248406F20B1012830D0B8
:1030A00002284ED13AE03E49086DFDF7FCFA06468B
:1030B000414801683046FDF7FEF805463848016F83
:1030C0002846FDF7A0F836490867886DFDF7EBFA4A
:1030D00005463348016F2846FDF77EFB07D230498D
:1030E000886DFDF7E0FA2E490867012048672C48F3
:1030F000006E2B49496E884202DB0120284948674F
:103100001FE02748C06D2649896E401A2449096E80
:10311000884202DC02202249486712E02049486DBB
:10312000FDF7C1FA0646244801683046FDF7C3F8AA
:1031300005461B48016F2846FDF7BAF8184908678D
:1031400000BF00BF1648046F2046FDF7FEFA074691
:1031500000221A4BFDF7C6F90546FDF721FB814613
:103160004846FDF7BFFA054600F068F90C48006EC6
:103170000B4900E012E0C96D884205DA0848006892
:103180000749C96C884208D100F0D2F90448C06CE4
:10319000034908604FF0FF30486700BF00BF6EE78B
:1031A00050000020737465705F636F756E74657294
:1031B000203D2025640D0A00200000200000F03F83
:1031C00010B501201D49C860086108460023D0E9F8
:1031D0000A219A1A73EB010013DA4FF48051184850
:1031E000FDF74EFF0121C802FDF7C4FF4FF4006157
:1031F0001348FDF747FF00201049486011A0FEF773
:10320000BDFF0E48D0E90A30002211469A1A8841C3
:1032100013DA4FF480510A48FDF734FF0121C80248
:10322000FDF7A8FF4FF400610548FDF72BFF0120D3
:103230000249486007A0FEF7A1FF10BD5000002022
:10324000000801407A68656E677A6875616E0D0ADC
:103250000000000066616E0D0A0000002DE9F05FBD
:10326000044600F065F95748C4640068A0420BD1D9
:10327000544890F8780038B900F05AF9214652A025
:10328000FEF77CFFBDE8F09F4E480068271A381E05
:1032900001DB014600E041424A4AD165002F01DCD2
:1032A000012000E0002047494860096D4900454A77
:1032B000D26D01FB02F0FDF704FA80460022484B74
:1032C000FDF710F9824600F00CF905460E463D491F
:1032D000886DFDF7F6F982462A463346FDF748FA2F
:1032E00002D22846314603E03649886DFDF7E9F9F8
:1032F0008046FDF70BFA334988650846806D4043E8
:10330000096D490090FBF1F02E4948660846806D32
:103310004043496D490090FBF1F02A498866084610
:10332000406E896E08442749C96D88420ADC2548E9
:10333000C06D2449496E401A2249896E401A2149BC
:10334000C86615E01F48C06D1E49496D48431D49B8
:10335000096D1C4A526D114490FBF1F01949486601
:103360000846C06D496E401A164988660020C86636
:103370001448C06DC117134AC2E90A010120114661
:10338000C860002008660867486701200861C861B6
:103390000846406828B94FF480511248FDF770FE86
:1033A00004E04FF480510F48FDF76CFE4FF40061CC
:1033B0000C48FDF767FE0121C802FDF7DBFE00BFE8
:1033C00060E7000050000020416C72656164792064
:1033D0006174207461726765743A2025640D0A0077
:1033E0000000F03F0008014010B501200D4981F8B0
:1033F000780040210C48FDF73AFE012804D100F086
:1034000097F8002007490860064890F878000128DE
:1034100007D140210448FDF72AFE10B90348FFF701
:103420001DFF10BD50000020000C0140F6E5FFFF1D
:1034300010B50446A0B2FDF76DFC10BD2DE9F041BA
:1034400005461E4F0026002D05DC00211C48FEF716
:10345000D5FBBDE8F081B7FBF5F0441E06E0701C1B
:1034600086B205FB06F0B7FBF0F0441EB4F5803FD2
:1034700003D34FF6FF708642F1DBB4F5803F00D3F3
:10348000E7E700210E48FEF7B9FB00210C48FEF7E4
:10349000A3FB0B4828300680011D0C80C4F34F00AD
:1034A00007493431088001210548FEF795FB0121C9
:1034B0000348FEF7A3FB00BFCBE7000000A24A04CD
:1034C000002C014070B506460C46154625B9A1B240
:1034D0003046FDF7D5FD03E0A1B23046FDF7D2FD41
:1034E00070BD2DE9F04106460F46FDF7C3FA041EF4
:1034F0000D4618BF0120284320F00040C0F17F6036
:1035000000F1E040C00F0ED0301C18BF012038433E
:1035100020F00040C0F17F6000F1E040C00F04BF28
:103520000120FEF74FFE20462946BDE8F08100004D
:1035300010B54FF400610748FDF7A2FD00214FF4DC
:103540000060FDF717FE0020034908610866086760
:1035500010BD0000000801405000002010B586B0EA
:103560000446012144F20400FDF704FE4FF400700C
:10357000ADF8140003208DF8160018208DF8170000
:1035800005A91C48FDF7E8FC4FF48060ADF8140075
:1035900004208DF8170005A91648FDF7DDFC25204D
:1035A0008DF8000003208DF801008DF80200012045
:1035B0008DF803006846FDF789FD01940020ADF801
:1035C0000800ADF80A00ADF80C00ADF810000C20B2
:1035D000ADF80E0001A90848FEF758FD012240F29F
:1035E00025510548FEF72DFD01210348FEF7E6FCB5
:1035F00006B010BD000801400038014000404040C6
:1036000040404040404041414141414040404040B5
:103610004040404040404040404040404005020261
:103620000202020202020202020202020220202020
:10363000202020202020200202020202020290907C
:10364000909090901010101010101010101010107A
:1036500010101010101010100202020202028888CE
:1036600088888888080808080808080808080808DA
:1036700008080808080808080202020240000000C2
:10368000FD350008A43600080000002050000000AE
:10369000A4210008F4360008500000205005000066
:1036A000B4210008000000000000000000A24A044D
:1036B00000000000000000000102030406070809E2
:1036C000000000006F12833A0000000000000000BC
:1036D00000000000000000000000000001020304E0
:1036E000010203040607080902040608000000009E
:0436F00000000000D6
:0400000508000145A9
:00000001FF
